:0200000046298F
:020008002829A5
:04000C000D08820752
:100010000034FF340D0882070234FF340D088207D4
:1000200002340234FF340D088207023402340234F1
:10003000FF340D0882070234023402340234FF34E4
:100040000D08820702340234023402340234FF34D1
:100050000D088207023402340234023402340234BE
:10006000FF340D08820702340234023402340234B1
:1000700002340234FF340D088900831608148312F9
:10008000080808000D088207093402340034FF34E0
:100090000D088207003407340F340034FF340D0894
:1000A00082070034183402340A343E340A343F34B0
:1000B00031340034FF34B620060807398207672838
:1000C0008C28922898289E28B128B128B128093078
:1000D000BC2000308D0085196B280D0889000608AA
:1000E00088008E008316081555308900AA308900D3
:1000F000881408118312851D7B280608FF3A03190E
:100100008428EA208D0A6B2803308E009000FF308F
:100110009500EA20B6208B2885198C2809308900A3
:10012000A4208A28851992280A308900A4208A28C8
:10013000851998280B308900A4208A2885199E28C3
:100140000C308900A4208A28060807398800831605
:10015000081555308900AA308900881408118312C7
:100160000800913095000B30BC20B1280130900080
:1001700085140221851008008C008D0103100C0DE0
:1001800082070620D8280A20D8280E20D828132035
:10019000D8281920D8282020D8282820D82831204D
:1001A000D8283B20D8284220D8284820D8284F20BB
:1001B0008E008E080319E628FF300E06031908008A
:1001C000EA208D0A02308F001521BE2804308F00EE
:1001D0001521E12803108E0C8E0803190800031C5A
:1001E000FA280330900001308F0085140221851019
:1001F0001521EA28013090008F0085140221851016
:100200001521EA2810089100150892000514B23053
:100210009300930B09290510B2309300930B0E291C
:10022000920B0629910B042908000F08910015086C
:1002300092001414B2309300930B1C291410B230A6
:100240009300930B2129920B1929910B1729080070
:100250009700030E9800990B402910309900A30ACB
:100260009B0B342906309B009A0B40292114160859
:100270009A009E0A1E081F02031D402901309E009D
:100280000B11180E8300970E170E0900073062003D
:100290008501860108306500FF30660085195B28FE
:1002A00001308A005329810164008B018B178B1662
:1002B00010309900A10109308900831608148312B7
:1002C0000808A0000B308900831608148312080860
:1002D0000319013EA2000A30890083160814831214
:1002E00008080319013E013E9F001F08220203185F
:1002F0008F210C3089008316081483120808862188
:1003000096009A0096218B136300000082070A343E
:100310000C340F3414341E34243430343C34190873
:100320000239031D8514031985108F2901309E00A1
:100330001E082206031D9829A3010516231C9E29C9
:10034000051506309B0021105A30950000308A00B8
:100350002008B2291A080B3C0318B7291B08063CD1
:10036000031DAE290A30BC202008BC20AA291B0886
:10037000063C031DB7293C3095000930BC200830ED
:10038000BC2001308A00211CC329A301231CC629DB
:100390000A3089008316081483120808013A0319E9
:0C03A000982905112318D229051298296C
:02400E00F13F80
:104200000A000F0015000600FF00FF00FF00FF007E
:0A421000FF00010005000100070097
:00000001FF
